:020000020000FC
:1000000019C094C01895ECC0DDC01895D7C01895DC
:10001000FCC000C118951895189518951895189555
:10002000ECC01895189542423133205374617274B4
:10003000204F4B3704E00EBF0FE50DBF01E00FBBB3
:100040000FEF0EBBE09A0DB301BF00E008BB00E06C
:1000500007BB00E005BB0CE204BB00E002BB08E309
:1000600001BB02E003BF02E00EBD77278827992776
:1000700090937600909377009093BF009093240123
:10008000BB27A0E600270D93A438E8F39460FF2473
:100090002BD302E3B02E10D1C19AD5D194FDFDCF60
:1000A0000CE002E192FD08E4302E06EF202E00273E
:1000B000C02ED02E009381000093820005E108BF7E
:1000C00009BF0FEF02BF002705BD002705BD04BD16
:1000D000106408B7012B08BF09B7006409BF789402
:1000E00003E005BF00E40BBF2AE083FFFECF092D2C
:1000F0001A2D877F0C541440B8F72A95B1F7F8945D
:10010000A2D1A1D1C19893FD9ED17894F9E07F7DD1
:100110007061C3D1DDD292D2379800B7086000BFBA
:1001200000917700046000937700F3C31FB6442763
:100130004BBF45B740FF1EC0829B3CC042E045BF5D
:100140004CB55DB5742E852E9F7B60917300461B68
:1001500060917400560B483A61E6560730F448390E
:100160006AE3560710F0906425C0BB2018F587FF9E
:10017000BA9420C082991EC043E045BF83FD1AC0D7
:100180004CB55DB5409373005093740096FF12C058
:100190009F7B47195809942EA52E483968E05607C9
:1001A00020F7403263E0560700F388604B2D42335E
:1001B00008F4B39450E45BBF1FBE18951FB67E7F52
:1001C0001FBE18951FB6442775FD939874FDAA9815
:1001D00074FD03C075FD01C0AD9845BD1FBE1895E7
:1001E0001FB642B344FD04C0949A959AAB9A03C0DB
:1001F00094989598AB981FBE18951FB645B3477C49
:1002000045BB4427642E1FBE18951FB643948068D3
:100210001FBE18951FB676FD30C0422D562D5417BF
:1002200088F43A94C1F452E192FD58E4662D641BBF
:10023000603328F06695669566956695560F352E5F
:100240004A9508C041F03A9431F458E092FD52E4E6
:10025000352E4395242E706474FF03C081FFAB9844
:1002600007C075FF03C081FF949802C081FF959875
:10027000422D4C59409542BF1BC0422D42BF7F7B4F
:1002800074FF03C080FFAB9A07C075FF03C080FFF7
:10029000949A02C080FF959A4C3918F482608E7F40
:1002A00007C0463F18F08D7F816002C08D7F8E7F32
:1002B00091FD81601FBE1895F89400279860C29A3E
:1002C00000000000000000000000B2999860B29B9E
:1002D000977FC29800B7077F00BF01E007B90027EA
:1002E00041E055E0076006B9379AC1D0FF24369A3D
:1002F0003699FECF04B115B1369AF39415E0F11694
:10030000B9F7FF24369A3699FECF04B115B1FF2014
:1003100039F4FF24F39410936A0000936B00F2CF3A
:1003200030916A0020916B00201B310B90F3442721
:10033000552730916A0020916B00020F131F451F53
:1003400046951795079510936A0000936B00F394F8
:1003500015E0F116B9F6FF2437980027076006B9B3
:100360000027016407B900916B0010916A00FF2417
:1003700093FD03C022E330E002C024E830E0F394B0
:10038000021B130BE0F7FA9493FD03C010E002E3A5
:1003900002C010E008E9222733274F2D200F311F1C
:1003A0004A95E1F700916B0010916A00201B310B18
:1003B00008F4F394F092700093FD05C010E000E2A1
:1003C00050E045E104C010E008E650E049E522278E
:1003D0003327200F311FFA94E1F720936C003093FC
:1003E0006D0022273327F0907000240F351FFA94F8
:1003F000E1F720936F0030936E0005EC10E0209140
:100400006C0030916D00311720F400936C00109354
:100410006D000027056006B93798FF2400B7086013
:1004200000BF23EB30E093FD04C020916F003091BA
:100430006E0000916B0010916A00021B130B08F014
:1004400008959460089510E8002702BF939A959A42
:1004500002B70032E9F79398959828E0002702BF89
:1004600002B70F3FE9F72A95C9F71A9569F710E81F
:1004700028E0002702BF02B70F3FE9F72A95C9F726
:100480001A95B1F7089530E03BBF30E03EBD32E051
:100490000CB51DB5242D3EBD0895F5DF30E43BBFFE
:1004A000009360001093610020936200C09163008C
:1004B000D0916400E09165000C1B1D0B2E0B34E005
:1004C0002695179507953A95D9F7C02FD12FE22F8A
:1004D0002223A9F410937200112329F0EE2408526C
:1004E000134268F40EC0EE2011F41FEFE12E122D1E
:1004F000159515951A5C011720F4C12F02C0E8D09C
:1005000032C0C0936600D093670092FD1EC0022DDA
:1005100000950535D0F00C2F1D2F169507951695D3
:10052000079516950795169507953327262D20953F
:1005300033952695E9F73A95532E22273327200F36
:10054000311F5A94E1F7C20FD31F92FD08C0D69510
:10055000C7950C2F1D2F16950795C00FD11FC0935F
:100560006800D093690000916000109161002091B3
:100570006200009363001093640020936500089567
:1005800083FF02C002D08ED0089583FF24C0092DBE
:100590001A2D877F0C54144010F40027112716954C
:1005A00007951695079516950795202F0456104028
:1005B00008F024E692FF0EC02A3060F02F2F2A3078
:1005C00018F411272AE0210FF39406E90F1510F013
:1005D0002395FF24F22F089587FF19C08F7708C055
:1005E00072FF06C07B7F4C2D453098F4C39403C046
:1005F000CC2009F0CA9471FF07C07D7FC1984D2DB2
:10060000443628F4D39403C0DD2009F0DA944AD0AC
:1006100008956AD0F8940ECD7160C0916600D091B3
:10062000670031DFC00FD11F05E409BFDBBDCABDC4
:1006300005E509BF30E43BBF70FDFECF379800B73A
:10064000086000BF71601FDFC0EBD6E30C0F1D1FF9
:1006500025E429BF1BBD0ABD25E529BF30E43BBF0A
:100660000895716010DFC0916800D09169000C0F8F
:100670001D1F25E429BF1BBD0ABD25E529BF30E4A8
:100680003BBF82FD0ADF84FD80DF85FDA5DF77FDAE
:100690004CD286FD2BD292FF02C097FD089570FDCB
:1006A000FECF08950F2F0D1908F409E01091720084
:1006B000183028F012E3011740F0012F06C0143063
:1006C00020F014E6011708F0012F0095602E089520
:1006D00006EF202E08E000937200C8E2D3E2C09338
:1006E0006600D0936700089506EF602E00E09498AE
:1006F0009598AB989398AD98AA9802E1302E8160B6
:100700009D7F8D7F9460089504E00A95F1F7089528
:10071000002705BD04BD08B710641F7708BF09B7DF
:1007200000640F7709BFE0DF08959B7F70FD03C071
:1007300027DFD39408C0459BF8CFE6DF459BF5CF74
:1007400070688FDF7F77AD98000000000000000028
:1007500080FF939A07E007B95FDF70FD02C0D39472
:1007600008C0459BFACFD0DF4599F7CF806179DF8C
:100770008F7E04E509BF7F7D7F7E81FD02C076FD0F
:1007800003C0AB9880FF959A05E509BF00E007B963
:1007900043DF70FD02C0D39406C0459BFACFB4DF9F
:1007A000459BF7CF5EDF939800000000000000003B
:1007B00080FFAA9A06E007B92FDF70FD02C0D3942C
:1007C00008C04599FACFA0DF4599F7CF806449DF8B
:1007D0008F7B04E509BF70627F7E81FD02C076FDDC
:1007E00003C0959880FF949A05E509BF07E007B913
:1007F00013DF70FD03C0D394EFDE08C0459BF9CF33
:1008000083DF459BF6CF80622CDF8F7DAA980000A6
:1008100000000000000080FFAD9A00E007B9FCDE98
:1008200070FD02C0D39408C04599FACF6DDF459999
:10083000F7CF846016DF8B7F04E509BF7F7D706191
:1008400081FD02C076FD03C0949880FFAB9A05E558
:1008500009BF06E007B9E0DEBB2061F091FD08C0EA
:1008600080FF06C055DF9E7F946002E3B02E51C02A
:100870009B7F5BCFF894DECB777F00271127222761
:1008800030E106E007B9002700000000459B016049
:10089000102F2A9549F0459B1160000045991E7F55
:1008A0001017B9F3786008953A9599F708959598D7
:1008B000AB989498AD98AA98939873FD089594FD79
:1008C00008959061F894AA9A00000000949A959A6D
:1008D0000027112700000000000000000395D1F759
:1008E000000000000000959800271127000000007C
:1008F0000395E1F700000000AA98959894980000ED
:1009000000000000000000000000000000007894DB
:10091000089536DE946090689F7E0FEFE02EDD2410
:10092000ABDF1AEF73FD1FEFE12E06E007B9009170
:1009300082000093810073FD06C0002700938100B0
:1009400080FDE7CF00C070FD02C0906206C0459BED
:10095000FACFDADE459BF7CF84DEAD9800000000C9
:1009600080FF939A07E007B99D7F0E2D0D3F29F078
:100970000C3F19F00B3F09F001C092604DDE0E2DC7
:10098000083C08F49F7770FD02C0906208C045994A
:10099000FACFBADE4599F7CF806163DE8F7E04E53A
:1009A00009BF7F7D7F7E81FD02C076FD03C0AB98CD
:1009B00080FF959A05E509BF00E007B92DDE70FDBF
:1009C00002C0906206C0459BFACF9EDE459BF7CFE2
:1009D00048DE93980000000080FFAA9A06E007B95D
:1009E0001BDE70FD07C090620E2D043609F444989A
:1009F000C7DD06C04599F5CF87DE4599F2CF31DED8
:100A000004E509BF70627F7E81FD02C076FD03C0F0
:100A1000959880FF949A05E509BF07E007B99D7F87
:100A20000E2D013051F0EA940E2D043029F00330E0
:100A300019F0023009F001C09260EEDD70FD02C0D5
:100A4000906208C0459BFACF5FDE459BF7CF80627E
:100A500008DE8F7DAA980000000080FFAD9A00E0BC
:100A600007B90E2D18EC73FD16E9011708F49B7FEA
:100A7000D3DD70FD08C0906273FD03C00E2D043BF2
:100A800008F40BDD08C04599F4CF3EDE4599F1CF5F
:100A90008460E7DD8B7F04E509BF7F7D706181FDA8
:100AA00002C076FD03C0949880FFAB9A05E509BFAC
:100AB00006E007B9B1DD91FD02C080FD2ACF0091AB
:100AC000760095FD002703950093760095FDD3945D
:100AD0009F7D023018F4BB2041F034CF9B7F9F777D
:100AE000EE244EDD02E003BF20CEC4CE089586FF83
:100AF000089507B10093710004E007B900B7077FBC
:100B000000BF379A00000000369A3699FECF8F7BDF
:100B100004B115B1043108F074602091710027B957
:100B2000379820B7286020BF089577FF089507B150
:100B30000093710001E007B900B7077F00BF379A43
:100B400000000000369A3699FECF04B115B17F77C8
:100B50002091710027B9379820B7286020BF2091D5
:100B60006C0030916D00201B310B80F07260C19AD7
:100B70008D7F23EB30E093FF04C020916F00309114
:100B80006E00201B310B10F005E0D00EFF240895FD
:100B9000A895F8941FBB0EBBE09AE099FECF0DB369
:100BA00078940895A895F894E199FCCF0EBB1FBBEB
:0A0BB0002DBBE29AE19A78940895B3
:00000001FF
